:1000000019C033C032C031C030C02FC02EC02DC087
:100010002CC02BC02AC029C028C027C026C025C09C
:1000200024C023C022C021C020C01FC01EC01DC0CC
:100030001CC01BC011241FBECFEFD4E0DEBFCDBF5C
:1000400011E0A0E0B1E0E6E1F1E002C005900D9220
:10005000A030B107D9F711E0A0E0B1E001C01D92D6
:10006000A030B107E1F721D054C0CACF9093C500AA
:100070008093C400E1ECF0E080818860808380811F
:10008000806180830895982F8091C00085FFFCCF08
:10009000992309F49FE59093C60008958091C000CC
:1000A00087FFFCCF8091C60008958FEF84B98FE35E
:1000B00087B98EE38AB984E190E09093C50080937C
:1000C000C4008091C10088608093C1008091C1000C
:1000D00080618093C10078945FE54DE09AE002C0B2
:1000E0002F5F3F4FA89521153105D1F78091C000B2
:1000F00085FFFCCF5093C6008091C00085FFFCCFE8
:100100004093C6008091C00085FFFCCF9093C6004D
:06011000E7CFF894FFCFD9
:00000001FF
